:020000040007F3
:10800000588F0020D5830700DD830700DF8307003A
:10801000E1830700E3830700E58307000000000019
:10802000000000000000000000000000C183070005
:10803000E983070000000000EB830700ED830700E1
:10804000EF830700EF830700EF830700EF8307004C
:10805000EF830700EF830700EF830700EF8307003C
:10806000EF830700EF830700EF830700EF8307002C
:10807000EF830700EF830700EF830700EF8307001C
:10808000399B0700EF830700EF830700EF830700AA
:10809000EF830700EF8307009D970700EF8307003A
:1080A000EF830700EF830700EF830700EF830700EC
:1080B000EF830700EF8307000000000000000000CE
:1080C000EF830700EF830700EF830700EF830700CC
:1080D00029970700EF830700EF83070000000000E7
:1080E0000000000000000000000000000000000090
:1080F0000000000000000000000000000000000080
:10810000000000000000000000000000000000006F
:10811000000000000000000000000000000000005F
:10812000000000000000000000000000000000004F
:10813000000000000000000000000000000000003F
:10814000000000000000000000000000000000002F
:10815000000000000000000000000000000000001F
:10816000000000000000000000000000000000000F
:1081700000000000000000000000000000000000FF
:1081800000000000000000000000000000000000EF
:1081900000000000000000000000000000000000DF
:1081A00000000000000000000000000000000000CF
:1081B00000000000000000000000000000000000BF
:1081C00000000000000000000000000000000000AF
:1081D000000000000000000000000000000000009F
:1081E000000000000000000000000000000000008F
:1081F000000000000000000000000000000000007F
:10820000DFF80CD000F038F90048004785AA0700D5
:10821000588F002030B450E8012F93B2C489234412
:108220008489A34228BF1B1B0489A34202BFBFF35A
:108230002F8F002007E0C3EA020340E80134002C3E
:10824000E9D14FF001000A6030BC704750E8012FBF
:10825000C2EA024240E801210029F7D1704730B458
:1082600050E8022F1FFAA2F3C488A34202BFBFF353
:108270002F8F00200DE0C48923448489A34228BFA6
:108280001B1BC2EA034340E80234002CE8D14FF044
:1082900001000A6030BC704750E8022FC2EA224257
:1082A00040E802210029F7D17047034653E8022F26
:1082B000D988B2EB324F4FF0000017BF92B241EABB
:1082C000014142EA014104E05A68B2EB324F08BF73
:1082D000012043E80212002AE8D1704730B4044676
:1082E00054E8000F0D4644E80053002BF8D1156008
:1082F00030BC704730B4044654E8000F40EA010532
:1083000044E80053002BF7D1156030BC704730B4FF
:10831000044654E8000F00EA010544E80053002B2E
:10832000F7D1156030BC704730B4044654E8000FF4
:1083300080EA010544E80053002BF7D1156030BCFA
:10834000704730B4044654E8000F00EB010544E8E0
:108350000053002BF7D1156030BC704730B4044691
:1083600054E8000FA0EB010544E80053002BF7D1BF
:10837000156030BC704770B404464FF0000054E8FC
:10838000006F0D68AE4207BF44E80023012044E8B7
:1083900000630E60002B1CBF0020F0E770BC70472C
:1083A00030B4044654E8000F88422CBF451A0546F5
:1083B00044E80053002BF5D1156030BC7047000035
:1083C0001EF0040F0CBFEFF30880EFF3098003F0F9
:1083D0005FBE00000648804706480047FEE7FEE70C
:1083E000FEE7FEE7FEE7FEE7FEE7FEE7FEE7FEE765
:1083F000A197070001820700202A04DB203A00FA37
:1084000002F1002070479140C2F1200320FA03F3EB
:1084100019439040704740EA01039B0703D009E0ED
:1084200008C9121F08C0042AFAD203E011F8013B60
:1084300000F8013B521EF9D27047D2B201E000F8B9
:10844000012B491EFBD270470022F6E710B51346F8
:108450000A4604461946FFF7F0FF204610BD30B526
:1084600004460020034600E05B1C934203D2E05C1C
:10847000CD5C401BF8D030BD064C074D06E0E068EF
:1084800040F0010394E8070098471034AC42F6D35B
:10849000FFF7BAFE5CDE07007CDE07002DE9F04343
:1084A0008BB08046129D15F9046B009614461F464A
:1084B00089462B4602A81146424600F0BAFC02A8A3
:1084C0000146129A00F0A5FC4046414602AA129BC2
:1084D00000F08FFC2046214602AA129B00F089FC86
:1084E0002B46384639464A46009600F0A2FC02A8C0
:1084F0003946129A00F08DFC02A8014642462B46EE
:10850000009600F096FC02A8014622462B460096F3
:1085100000F08FFC2046214642462B46009600F094
:1085200088FC484649462246129B00F062FC2046E1
:10853000414602AA2B46009600F07BFC384639469D
:108540002246129B00F055FC384639464A462B46D7
:10855000009600F06EFC204602A9324600F033FE81
:108560000BB0BDE8F083F0B589B01C4607460E4657
:108570001546684611461A4600F04BFC3846394607
:108580006A46234600F035FC684669462A4623467B
:1085900000F02FFC304631466A46234600F029FCA5
:1085A00009B0F0BD1AB1013A8B5C8354FAE7704709
:1085B0002DE9F0478846B3F902101F460825CB1D68
:1085C000202493FBF5F51F31954291FBF4F44FFA0B
:1085D00084F928BF15460646494600F075FA2A4632
:1085E00030464146FFF7DEFFB7F90230ED009D420D
:1085F00020D9ED1A06EB840100228E420AD251F8EE
:10860000040D20FA05F313430B60C5F1200300FAB3
:1086100003F2F2E72437384631464A4600F060FA62
:10862000012807D0304631463A464B46BDE8F04770
:1086300000F01EBFBDE8F0872DE9F04793F9006018
:1086400092B004468946104631461546984600F0D9
:1086500071FA002840F0978002A84946424600F08F
:10866000D8FB43460AA8214602AA00F0C2FB02A892
:108670000146424600F0CDFB4346484649462A465D
:1086800000F0B7FB08F1040728462946424600F0EF
:10869000C0FB204621462A463B46009600F0F8FAE9
:1086A000284629462A463B46009600F0F1FA28461D
:1086B00021462A463B46009600F0BBFB2046214659
:1086C0002A46434600F095FB2846214622463B4673
:1086D000009600F0DDFA20463B46009621462A46E9
:1086E00000F0D6FA2368DB07204613D5334621462F
:1086F0003A4600F0BDF931468246204600F056FD6C
:1087000006F18043013B54F8230040EACA7044F864
:10871000230002E0314600F049FD2846214642464A
:1087200000F077FB284629460AAA3B46009600F04F
:1087300080FB284629460AAA3B46009600F079FBB2
:108740000AA801462A463B46009600F072FB2046E6
:1087500021460AAA434600F04CFB02A802463B46CB
:108760002146009600F065FB20462946324600F07F
:108770002AFD28464946324600F025FD484602A912
:10878000324600F020FD12B0BDE8F0870048704787
:10879000ACDD07002DE9F04FEFB01E46789C059048
:1087A00023780493B4F9023092461F33202293FBBE
:1087B000F2F3DBB206939DF9187094F9012007F1EA
:1087C000FF3926AB002543F829506EAB03EB890334
:1087D0004EA88B46314643F8805C43F8605CFFF757
:1087E000E1FE94F9012056A8B118FFF7DBFE9DF9D0
:1087F00010604EA8314600F09DF98046002840F0F8
:108800002F8156A8314600F095F90546002840F022
:10881000258104F1240840464EA93A4600F060F94B
:10882000012840F01D81404656A93A4600F058F90B
:108830000128089040F014813B461EA856A94246E4
:1088400000F03FFA0DF1380C604659465246234677
:108850004CF82950CDF80CC0FFF7AAFEDDF80CC08B
:108860000097604661461EAA4346CDF824C00DF528
:10887000BC7900F0ACFA4346009716A84EA91EAA90
:1088800000F0A5FA48463246059900F09CFCB3007A
:10889000039309EB030B039A059B5846991832463C
:1088A00000F091FC04F144031946324636A80793C0
:1088B00000F089FC04EB860132463EA8443104F105
:1088C000040A00F080FC494600961EA836AA5346CA
:1088D00000F0AFFA4A465B4636A83EA90094FFF77F
:1088E000DDFD1EA801463346524600F0EAF91EAAF5
:1088F000484659462346FFF736FEDDF824C0079B5D
:108900000B936046059B0C933946CDF814C00A952D
:10891000CDF8349000F028FC3946054616A800F042
:1089200023FCA842B8BF284685B2DDF814C06F1EEC
:108930003FB26046394600F0CBFD394610F10009E0
:1089400016A818BF4FF0010900F0C2FD002814BF9F
:108950000223002343EA09090DF1280B32465BF894
:10896000297026A8394600F02EFC039B3246F918E0
:108970002EA800F028FC31461EA800F0A5F8023D04
:10898000089B1E93AEB237B2002F44DB23461EAACB
:10899000D4F8A45026A82EA9A84739460EA800F05E
:1089A00097FD3946051C16A818BF012500F090FD5B
:1089B000002814BF022300231D430AAB53F825707F
:1089C00037B39DF9105036A839462A4600F0FBFB14
:1089D000039B3EA8F9182A4600F0F5FB36A83EA9ED
:1089E0001EAA2346FFF7BFFD46A826A936AA53466E
:1089F000009500F01EFA36A83EA926AA2EAB0094D8
:108A0000FFF74CFD1EA8014646AA234600F0F1F9E7
:108A1000013EB6B2B7E79DF910501EA80146524676
:108A20002B4600F04EF9234626A82EA91EAAFFF7D2
:108A30009AFD9DF91840404626A9224600F050F8BC
:108A4000012805D026A801464246234600F010FD25
:108A500026A84EA92A4600F058F802E0404600E059
:108A600028466FB0BDE8F08F000000000000000055
:108A7000C3F10803DB0070B501330446002003A5F1
:108A80005B1920C940CAAD1920C4184720C940CA83
:108A9000754120C420C940CA754120C420C940CABC
:108AA000754120C420C940CA754120C420C940CAAC
:108AB000754120C420C940CA754120C420C940CA9C
:108AC000754120C4404170BD10B5002253B28B42A5
:108AD00005DA1BB2002440F823400132F6E710BD4E
:108AE00010B5013AD2B253B2002B09DB1BB250F8D9
:108AF000234051F823309C4204D8F2D2FF2002E0F8
:108B0000002000E0012040B210BD013A30B5D2B2E1
:108B1000002453B2002B09DB1BB2013A51F8235059
:108B200050F823306B401C43D2B2F2E7B4FA84F021
:108B3000400930BD10B500231A465CB28C4204DAFD
:108B400050F8244001332243F7E7B2FA82F040099B
:108B500010BD00002DE9F043A3B09846019112AB7F
:108B60004146074610469146009300F0FDFAC0EBDF
:108B7000881086B2454C33B21C40002CBEBF04F1B5
:108B8000FF3464F01F040134202593FBF5F5EDB2AA
:108B90006DB2A4B202A8294624B2FFF795FF28B20D
:108BA00002AB002C03EB800010DD0022134643458E
:108BB00010D259F8235005FA04F10A4340F8232053
:108BC000C4F1200225FA02F20133F0E74946424699
:108BD00000F0F9FA0FFA88F502AB4FEA45090124D3
:108BE00003EB8505330444D40022114653B24B45B0
:108BF00022DA0DF1880E0EEB840E0DF1880C18B2FE
:108C00005EF888EC0CEB83035EF820E053F8803CC0
:108C1000C3EB0E035B1A734502D08CBF0121002108
:108C2000C4F1010E0DF1880C0CEB8E0E01325EF8D2
:108C300088EC4EF82030D9E7621A544202A8414627
:108C4000544100F0B3FA22AA08F1FF3302EB830388
:108C500002EB8802284652F8801C53F8802C013E13
:108C600042EAC172414643F8802CB6B200F09EFA47
:108C7000B8E722AB03EB8404384654F8881C42461C
:108C800000F0A1FA23B0BDE8F08300BF1F00008010
:108C900070B59DF910401D4623460646FFF7E8FED5
:108CA00030B9284631462246FFF71AFF012807D07F
:108CB000304631462A462346BDE8704000F0D8BB16
:108CC00070BDF0B50646A1B00F46084619461546D8
:108CD0001C46FFF72FFF20B130462146FFF7F4FE78
:108CE00073E068463946224600F06DFA08A8294626
:108CF000224600F068FA10A82146FFF7E5FE01239E
:108D000018A821461093FFF7DFFE684608A92246FF
:108D1000FFF7E6FE002853D0009BDA0704D468462C
:108D2000214600F043FA26E0089BDB0704D408A89C
:108D3000214600F03BFA3DE000281EDD08AA23464C
:108D40006946684600F094FB6846214600F02EFA1A
:108D500010A818A92246FFF7C3FE002805DA10A8BC
:108D600001462A462346FFF783FE10A8014618AAAB
:108D7000234600F07DFB10A81DE008A86A462346A4
:108D8000014600F075FB08A8214600F00FFA18A86C
:108D900010A92246FFF7A4FE002805DA18A801460C
:108DA0002A462346FFF764FE18A8014610AA234668
:108DB00000F05EFB18A82946224600F06BFCA4E7F1
:108DC000304610A9224600F0FEF921B0F0BD70B582
:108DD00090B006469DF950401D466846234600F077
:108DE0003AF8304669462A462346FFF7B3FE10B0EC
:108DF00070BD30B51C4691B0054693F90030684609
:108E000000F029F8D4F8AC3028466946984711B0EC
:108E100030BD30B5144691B0054692F90020684641
:108E200000F0DEF9D4F8AC3028466946984711B016
:108E300030BD70B59DF910401D462346064600F032
:108E400017FB38B1304631462A462346BDE870400C
:108E5000FFF70EBE70BD2DE9F04F08B4F8CA04B498
:108E600051F8042BA3FB028940F8048B4FF0000A51
:108E7000E4FB629A4FF0000BE5FB62AB4FF0000C95
:108E8000E6FB62BC4FF0000EE7FB62CE51F8042B0C
:108E90004FF00008E3FB628940F8048BE4FB629A20
:108EA000E5FB62ABE6FB62BCE7FB62CE51F8042B4C
:108EB0004FF00008E3FB628940F8048BE4FB629A00
:108EC000E5FB62ABE6FB62BCE7FB62CE51F8042B2C
:108ED0004FF00008E3FB628940F8048BE4FB629AE0
:108EE000E5FB62ABE6FB62BCE7FB62CE51F8042B0C
:108EF0004FF00008E3FB628940F8048BE4FB629AC0
:108F0000E5FB62ABE6FB62BCE7FB62CE40F8049B8C
:108F100040F804AB40F804BB40F804CB40F804EB45
:108F20000CBC052B00F01E810C68A0F11400A1F10F
:108F30001401A2F1140252F804EB4FF0000550F8AE
:108F4000046BE4FB6E5652F804EB50F8047BE4FB30
:108F50006E6752F804EB50F8048BE4FB6E7852F81D
:108F600004EB50F8049BE4FB6E8952F804EB50F8D4
:108F700004ABE4FB6E9AA0F1140052F8044B51F8D4
:108F800004EB4FF0000CE4FB6EC540F804CB51F845
:108F900004EBE4FB6E5640F8045B51F804EBE4FB91
:108FA0006E6740F8046B51F804EBE4FB6E7840F810
:108FB000047B51F804EBE4FB6E8940F8048B51F814
:108FC00004EBE4FB6E9AA0E80006062B00F0CA80D2
:108FD0000C68A0F11800A1F11801A2F1180252F8D2
:108FE00004EB4FF0000550F8046BE4FB6E5652F8AA
:108FF00004EB50F8047BE4FB6E6752F804EB50F886
:10900000048BE4FB6E7852F804EB50F8049BE4FB0D
:109010006E8952F804EB50F804ABE4FB6E9A52F8F8
:1090200004EB50F804BBE4FB6EABA0F1180052F85F
:10903000044B51F804EB4FF0000CE4FB6EC540F814
:1090400004CB51F804EBE4FB6E5640F8045B51F896
:1090500004EBE4FB6E6740F8046B51F804EBE4FBAF
:109060006E7840F8047B51F804EBE4FB6E8940F81D
:10907000048B51F804EBE4FB6E9A40F8049B51F822
:1090800004EBE4FB6EABA0E8000C072B6AD008B43D
:109090000C68A0F11C00A1F11C01A2F11C0252F805
:1090A00004EB4FF0000550F8046BE4FB6E5652F8E9
:1090B00004EB50F8047BE4FB6E6752F804EB50F8C5
:1090C000048BE4FB6E7852F804EB50F8049BE4FB4D
:1090D0006E8952F804EB50F804ABE4FB6E9A52F838
:1090E00004EB50F804BBE4FB6EAB52F804EB50F811
:1090F00004CBE4FB6EBCA0F11C0052F8044B51F809
:1091000004EB4FF00003E4FB6E3540F8043B51F8EC
:1091100004EBE4FB6E5640F8045B51F804EBE4FB0F
:109120006E6740F8046B51F804EBE4FB6E7840F88E
:10913000047B51F804EBE4FB6E8940F8048B51F892
:1091400004EBE4FB6E9A40F8049B51F804EBE4FB5B
:109150006EAB40F804AB51F804EBE4FB6EBCA0E846
:10916000001808BCBDE8F08F0139C9B24BB2002B22
:109170000BDA013111F0FF0315D059B201F1804330
:10918000013B50F82320002304E050F82330002B4B
:10919000EAD0EEE712B152080133FBE7481E03EBB9
:1091A000401080B200E0184600B2704700EB810129
:1091B0000023884206D251F8042D43EA52030B6083
:1091C000D307F6E7704730B5002463B2934206DA5E
:1091D0001BB2013451F8235040F82350F5E730BD5D
:1091E0002DE9F04FB1E8005E06B4AAFB09124FF07A
:1091F0000003EBFB69234FF00004ECFB69344FF0F4
:109200000005EEFB69454FF00006EBFB6A63ECFBE3
:109210006A344918524176415B41A9FB09784FF005
:10922000000949F1000918EB0108A0E88001AAFB38
:109230000A78574158EB0608A0E88001EEFB6A4522
:109240004FF0000A4AF1000A4FF00001ECFB6B14EA
:10925000EEFB6B454FF00002EEFB6C255FEA59090F
:109260004941644152416D4149F10009EBFB6B3AC0
:109270001AEB010AA0E80804ACFB0C6A66415AEB41
:10928000020AA0E84004AEFB0E6A6E415AEB090ADE
:10929000A0E8400406BC052A00F0E680A0F1140016
:1092A000A1F11401B1E8E043A5FB0E344FF0000535
:1092B000E6FB6E454FF00006E7FB6E564FF00007E9
:1092C000E8FB6E674FF00008E9FB6E784FF000098D
:1092D000DB1864416D4176417F4158EB080859F134
:1092E000000950F804CB13EB0C0350F804CB54EBFB
:1092F0000C0450F804CB55EB0C0550F804CB56EB9E
:109300000C0650F804CB57EB0C0758F1000859F144
:109310000009A0F11400EEFB0E89A0E8F803062A6C
:1093200000F0A280A0F11800A1F11801B1E8E04717
:10933000A5FB0E344FF00005E6FB6E454FF000062E
:10934000E7FB6E564FF00007E8FB6E674FF0000832
:10935000E9FB6E784FF00009EAFB6E894FF0000AD6
:10936000DB1864416D4176417F4158EB080859EBA9
:1093700009095AF1000A50F804CB13EB0C0350F81A
:1093800004CB54EB0C0450F804CB55EB0C0550F80F
:1093900004CB56EB0C0650F804CB57EB0C0750F8F7
:1093A00004CB58EB0C0859F100095AF1000AA0F15E
:1093B0001800EEFB0E9AA0E8F807072A54D0A0F197
:1093C0001C00A1F11C01B1E8E04FA5FB0E344FF0E9
:1093D0000005E6FB6E454FF00006E7FB6E564FF0CA
:1093E0000007E8FB6E674FF00008E9FB6E784FF06E
:1093F0000009EAFB6E894FF0000AEBFB6E9A4FF012
:10940000000BDB1864416D4176417F4158EB080841
:1094100059EB09095AEB0A0A5BF1000B50F804CB2F
:1094200013EB0C0350F804CB54EB0C0450F804CBB2
:1094300055EB0C0550F804CB56EB0C0650F804CB5A
:1094400057EB0C0750F804CB58EB0C0850F804CB42
:1094500059EB0C095AF1000A5BF1000BA0F11C005A
:10946000EEFB0EABA0E8F80FBDE8F08F00000000A7
:10947000C3F10803DB0070B50133002403A500BF6E
:109480005B1920C940CAAD1B20C0184720C940CA7B
:10949000B54120C020C940CAB54120C020C940CA3A
:1094A000B54120C020C940CAB54120C020C940CA2A
:1094B000B54120C020C940CAB54120C020C940CA1A
:1094C000B54120C06441B4FA84F0400970BD00BFCA
:1094D0004A11012301F01F0150F822008B4018406F
:1094E00070470000F0B50C4689B008220646FFF729
:1094F0006AFEE36A0393236B0493636B0593A36B88
:109500000693E36B0793002769466A46082368467B
:10951000029701970097FFF7ABFA314605466A4676
:1095200008233046FFF7A4FA236B0393636B04937D
:10953000A36B0593E36B0693054469466A460823CB
:1095400068460797FFF794FA314605446A460823B0
:109550003046FFF78DFA236A0093636A0193A36A8A
:109560000293A36B0693E36B0793054431466A4667
:1095700008233046059704970397FFF779FA636A43
:109580000093A36A0193E36AA26B0293636B039354
:1095900004920693E26B236A0592054407933146D1
:1095A0006A4608233046FFF763FAE36A0093236BA9
:1095B0000193636B0293236A0693A36A079305449E
:1095C00031466A4608233046059704970397FFF70C
:1095D0004FFF236B0093636B0193A36B0293E36BC9
:1095E0000393636A0693E36A07932D1A31466A462A
:1095F0000823304605970497FFF73AFF636B009303
:10960000A36B0193E36B0293236A0393636A04934E
:10961000A36A0593236B07932D1A31466A460823E4
:1096200030460697FFF724FFA36B0093E36B01938B
:10963000636A0393A36A0493E36A0593636B0793D6
:109640002D1A314630466A46082302970697FFF7DF
:109650000FFF2D1A16D5304631460D4A0823FFF765
:1096600007FA4519F7D410E0094831460822FFF7F8
:1096700037FA012809D030463146054A0823FFF75A
:10968000F7FE2D1A002DEFD0F5E709B0F0BD00BFB1
:10969000B0DD0700F8B5036813F0010506460F4674
:1096A000144605D001463A462346FFF7E1F9054640
:1096B00030462146FFF77AFD45B104F18042013A78
:1096C00056F8223043F0004346F82230F8BD2DE929
:1096D000F04115468AB00446884602A8002120229F
:1096E000FEF7B4FE2E780323204641462A462F1D5E
:1096F00076B20293FFF78DFB2046214602AA3B4635
:109700000096FFF796FB2046214642462B46FFF780
:1097100070FB00962046214605F184023B46FFF788
:10972000B7FA0AB0BDE8F0812DE9F041194E4FF4C7
:109730008271D6F8040130B11748C268521CC26069
:10974000304602F03DFB00254FF4A07707EB850182
:109750008AB23046B258BAB189B202F031FB0E4833
:10976000103000EB0514204603F076FF616819B154
:10977000204603F0F9FE07E0A16811B1204603F08E
:10978000F3FE206800B180476D1C022DDED3BDE8DA
:10979000F0810000004002407059002002F00CBC33
:1097A000F0B5D34AD3494FF080541368D4F8300150
:1097B0000978D4F83421451CC1F3031107D084463D
:1097C000164601270025BCF1060F04D013E003F074
:1097D000FF0C0E46F5E7032E05D0042E03D0052E10
:1097E00001D0062E07D1B4F82463DFF80CC3C6F30A
:1097F0000426CCF80060DEB2062E06D1032904D17F
:10980000DFF8FCC2BD4ECCF87460461C06D084461E
:109810004FEA0206BCF1060F04D013E003F0FF0C80
:109820000E46F7E7032E05D0042E03D0052E01D0F7
:10983000062E07D1D4F84462DFF8C8C2C6F3423618
:10984000CCF80060DEB2062E08D1032906D1AE4E58
:10985000D6F800C02CF0807CC6F800C0461C05D0AD
:1098600084461646BCF1060F04D014E003F0FF0C4A
:109870000E46F7E7032E05D0042E03D0052E01D0A7
:10988000062E08D14FF08046C6F80C51C6F810518C
:109890009C4E361F3560DEB2062E08D1032906D154
:1098A000DFF860C203260CF1640CCCF80060DEB275
:1098B000062E11D103290FD1DFF850C20526CCF8AE
:1098C0000060924E78363760904E083635600CF165
:1098D000040C3F26CCF80060461C05D08446164692
:1098E000BCF1060F04D087E003F0FF0C0E46F7E74B
:1098F000032E7CD0042E7FD0052E01D0062E7BD1E6
:10990000834E3668DFF80CC2CCF80060804E361DFE
:1099100036680CF1040CCCF800607D4E08363668D1
:109920000CF1040CCCF80060794E0C3636680CF162
:10993000040CCCF80060764E103636680CF1040C3E
:10994000CCF80060724E143636680CF1040CCCF87A
:1099500000606F4E18363668DFF8B8C10CF1200C85
:10996000CCF800606A4E1C3636680CF1040CCCF85A
:109970000060674E203636680CF1040CCCF80060AD
:10998000634E243636680CF1040CCCF80060604E4F
:10999000283636680CF1040CCCF800605C4E2C368E
:1099A00036680CF1040CCCF80060594E303636683D
:1099B000DFF860C10CF1400CCCF80060544E343636
:1099C00036680CF1040CCCF80060514E383636681D
:1099D0000CF1040CCCF800604D4E3C3636680CF1AE
:1099E000040CCCF800604A4E4036366800E003E0D4
:1099F0000CF1040CCCF80060461C05D084461646D9
:109A0000BCF1060F04D011E003F0FF0C0E46F7E79F
:109A1000032E05D0042E03D0052E01D0062E05D12D
:109A2000D4F858423C4E04F04F043460441C04D037
:109A300003461146062B02D010E0DBB2FAE70329F9
:109A400005D0042903D0052901D0062906D13349C0
:109A50000B68DB0702D06FF001030B6006280CD106
:109A6000032A0AD0042A08D0052A06D0062A04D1DF
:109A70002B48016841F48061016023487438016813
:109A800041F470010160BFF34F8FBFF36F8F4FF050
:109A90001021D1F80002002803DBD1F804020028CD
:109AA00022DA204A176020480368002BFCD01523D7
:109AB000C1F800320468002CFCD0C1F804320168FF
:109AC0000029FCD0156001680029FCD0BFF34F8F3E
:109AD0000D48F0380168154A01F4E0611143016056
:109AE000BFF34F8F00BFFDE7124911480860F0BD7A
:109AF000E00F00F0E80F00F0403501400DF0ADBA86
:109B000000C007403C050040FCED00E0105600405E
:109B10000404001020C50040E40E00400004004092
:109B20003C17004004E5014000E401400400FA0550
:109B30000090D003085A0020034808B500210160B6
:109B40000068009008BD00000001014002E008C864
:109B5000121F08C1002AFAD170477047002001E0A7
:109B600001C1121F002AFBD17047000001212028EB
:109B700003DA81400548014003E0402802DA20383A
:109B8000814009B10120704700207047FC06FFBDED
:109B9000800701D00020704701207047C3688B42C6
:109BA00006D811440069491E814201D8012070473E
:109BB0000020704730B585B00D46164C1621ADF823
:109BC00000101ECC0DF1040C8CE81E00124C02217A
:109BD000012221706270A0700320E0702171592071
:109BE0006071FE20A071694604F109007DDF002844
:109BF0000ED1BDF800002A46411CE17109212172F5
:109C0000BDF808100844ADF8080001A9034872DF48
:109C100005B030BD60DA0700405E0020A859002082
:109C200010B586B00624182208496846FEF7F3FBF3
:109C300069462046FFF7BEFF002805D1044C207876
:109C400074DF0121207873DF06B010BD70DA0700E1
:109C5000A859002070B5104CA66C656A01F096FA00
:109C6000216B08446A1A3144814200D10022082342
:109C700000F042FE06000DD101F088FA00222946CC
:109C800000F0B2FBA16A814203D10121A561C4E9C0
:109C90000701304670BD0000D875002002F03AFB85
:109CA00002F038FB2DE9F84F254C8146924660883A
:109CB0000E46814241D800274FF6FF788DF800709C
:109CC000684600F075F822786078A188884201DA49
:109CD000401C00E00020C0B2904204D19DF800007A
:109CE00000F08AF827E065786078884201DA401C45
:109CF00000E0002060709DF8000000F07DF8454510
:109D000019D0A068B9F1000F40F835A00DD066B1A8
:109D10006188E068324605FB01004946FEF77BFB9F
:109D2000A06800EBC500868002E000EBC5008780DC
:109D30000020BDE8F88F0420FBE70920F9E70000C8
:109D4000E859002010B50E4C03E0401C00E0002054
:109D5000207020786178814210D022786188E06894
:109D6000A36802FB010003EBC20153F8322089888B
:109D700090472078A1888842E9DAE6E710BD000024
:109D8000E859002030B5CB0008339DB293074FF05F
:109D9000000401D0072030BD044B9A602A44DA60E9
:109DA0005C701C7058809980002030BDE8590020FC
:109DB00030B5EFF3108172B60D4A9468012324B1D7
:109DC0000370002900D162B630BD93604FF0E023EC
:109DD000D3F88051074C25401560C3F88041D3F873
:109DE000844154605A17C3F8842100220270E8E7C6
:109DF0004C7D0020FC06FFBD0B498A68002A11D06B
:109E000000280FD1EFF3108072B60B684FF0E022FC
:109E1000C2F800314B68C2F8043100228A60002881
:109E200000D162B6704700004C7D002070B5164E20
:109E3000154856F8245F846CB168AC2901D024B170
:109E400011E0406B04442D1A05E001F0B3F904461B
:109E5000B068AC2807D12A46A4F580410B48FEF72C
:109E6000FEFA00280ED02A4621460848FEF7F7FAE7
:109E7000002807D001F004F829462046BDE87040CC
:109E800001F0BCBA70BD0000D8750020008007004A
:109E900030B504462C4995B04FF6FF70488001203C
:109EA0008DF812004FF65960ADF81000224604A953
:109EB0000120A8DF002844D1244B0FCB8DE80F00F0
:109EC000A11C684662DF00283BD120491C22603972
:109ED0000BA8FEF7A0FA1E4D142205F1C401A868D4
:109EE0001290A0788DF84A002868139006A8FEF713
:109EF00092FA12A8069013A807902088231D06AA9C
:109F00000BA9AADF00281CD11C2205F1D8010BA83F
:109F1000FEF781FAE8681290A0788DF84A00686828
:109F20001390142205F1F40106A8FEF774FA12A8A2
:109F3000069013A80790208804F10C0306AA0BA929
:109F4000AADF15B030BD0000A859002038DB07009B
:109F500030DA0700F0B585B0044614216846FEF7F4
:109F600073FA2078032308280BD12748C188491E9B
:109F700089B2C1808288002A3ED000293CD1C280AB
:109F800023702178607860228DF800208DF8011010
:109F90008DF802006078032101280AD00B2828D10F
:109FA00000F058FC8DF80300002000F05BFC042159
:109FB0001FE0207809281CD2DFE800F01B1B1B20C3
:109FC0001B1B051B2000D4E902706D46E91C666866
:109FD00003F04CFB044629193046C91C03F046FB2C
:109FE000044429193846C91C03F040FB2044C01C16
:109FF000C1B2684602F092FF05B0F0BDD4E901128B
:10A00000684602F07AFFF2E7A85900202DE9F041F6
:10A010001349034600208A68D4071ED0114CA3427E
:10A020001BD04888A0F57F43FF3B10D042F00402CC
:10A030008A60132176DF00280FD10B4EC8254FF41C
:10A040007A47741C3846A0476D1EFAD101E00878A3
:10A0500074DFBDE8F04101F04BBFBDE8F0810000C6
:10A06000A85900207CDE070040DA070038B5214CF3
:10A070000021227AD20701D0084638BDE0601E4890
:10A0800000F0AAFD0020009001F0C4F988B91B4837
:10A0900013DF70B901F056FF58B9684601F096FE1B
:10A0A00038B96946012001F09BFE10B9684601F0FD
:10A0B000E5FE0028E1D101F099FA30B1104801F035
:10A0C00089FAA06840F00200A06000F0E1FB0028DF
:10A0D000D3D10B481C30FFF7DBFE0028CDD1FFF7B2
:10A0E0009FFD0028C9D1A06840F00100A0600020B9
:10A0F00038BD0000A859002084DE0700008007005A
:10A10000605E002070B50446011D008800226F4D7E
:10A1100086B021287ED025DC13287CD018DC0128CD
:10A120007AD010285BD011284AD14FF6FF70688092
:10A13000287A400704D4FFF773FD08B1FFF7B0FD9C
:10A14000E96800293CD006B00220BDE8704008470D
:10A15000142878D01A2877D01F2831D16888091D93
:10A1600075DF62E0512870D02CDC222828D023280B
:10A1700062D0242824D0502822D1554D34F8060F1F
:10A18000A98888421CD1534800F0ECFC060017D087
:10A19000628904F10C01FEF73EF918224E49684627
:10A1A000FEF739F9049601956089ADF81400684608
:10A1B00001F064F9002803D03146464800F0F4FC71
:10A1C00006B070BD52287BD0552813D05628F7D141
:10A1D000A0790028F4D11321688876DF25E008886B
:10A1E0006880E96809B1012088473B4968887A3965
:10A1F00075DFE5E7E188F72914D28807B0F1404F11
:10A2000011D0C91F89B2481EC21700EB927222F00A
:10A21000030202E033E01CE036E0801A081A801DD9
:10A2200081B200E0F7216888B5DF0028C8D006B009
:10A23000BDE87040FFF734BD00920192A088002273
:10A24000694690DF18E034E03AE021E0FFF728FDAE
:10A25000B6E721486A46903842F60521806A0090A8
:10A2600002A801906888ADDF08B1FFF719FD00234F
:10A270001A46852168887FDF0028E7D1A0E7009291
:10A28000088869468FDFF7E70021688866DFCCE73A
:10A29000A079002894D021460D4802F053F80028F8
:10A2A0008ED006B004F10801BDE87040084801F006
:10A2B0003DBF0024088822462346214686DFB4E7B6
:10A2C000002308881A461946B1DFAEE7A8590020D6
:10A2D0007C5E002084DE0700C0DA0700007800F012
:10A2E0000100704713B90378012B01D001F0A1BA26
:10A2F000012070470022C32100F5187000F074B8E7
:10A300002DE9F043A1B00446DDE9289520200F4651
:10A31000209098461646782102A8FEF795F841212C
:10A320002046FEF791F8B7F8940006EB061107EB0C
:10A330008101B04201D991F8965025701DB3012DCD
:10A3400004D0022D0AD0032D13D116E00022494675
:10A35000404600F049F8C4F8010014E020A9601C50
:10A36000CDE900014B4642460A4902A800F036FEFC
:10A3700048B1002021B0BDE8F083B1F89820601CFE
:10A380009A31FEF748F84A464146204601F051FA14
:10A39000F0E7000058D8070010B500284FF0000083
:10A3A00006D004490870BDE81040034801F04AB9DE
:10A3B00000F0A8F96859002005A7070010B5436808
:10A3C0009C18446021B905E013F8010B01F8010B5A
:10A3D000521EF9D2012010BD0249CA6B4260096CBD
:10A3E00081607047D8750020F0B54FF0FF3622B17C
:10A3F0001268D24300230A4D0DE03246FAE7C45CEE
:10A4000062400824D70700D037462F4087EA52021F
:10A41000641EF7D15B1C8B42F1D3D043F0BD00002A
:10A420002083B8ED10B504460068401C07D02046D4
:10A4300002F04AFE2168814201D1012010BD0020B6
:10A4400010BD000010B50B4C90B0607800280ED104
:10A4500000F028FE20220849684600F043FE402311
:10A460006A460649064800F079FD0120607010B088
:10A4700010BD0000D859002004D80700847C0020BB
:10A4800070D80700F0B5146906468DB020681546EF
:10A49000271DE0B1022920D00A2000906B4609AAAE
:10A4A000304602F0F9FC00280FD009A901A8009A53
:10A4B00002F0E8FA01AE96E80F0005AE86E80F005C
:10A4C000236869683A4605A898470DB0F0BD0DB0FD
:10A4D0003046BDE8F04002F049BB6946304602F024
:10A4E000DBFA0028F1D0236869683A466846984745
:10A4F0000028EAD002980028F5D101987060012068
:10A50000E3E753689B7813F0C00303D0402B03D0DC
:10A510000020704700F002B8FFF7B4BF2DE9FF41FB
:10A520000B465168064614468878334D00F00F02FA
:10A5300010F0300055F8225006D0102806D0202800
:10A5400008D0302856D13EE022694DE061690120F3
:10A55000087047E0022B28D1042A26D84FF00108C2
:10A5600069463046676902F097FA00281AD009E078
:10A570000B89226903FB00226846A84770B138881E
:10A58000401C3880029820B1616838884A8990421E
:10A59000EED301987060029860BB02E04FF00008B3
:10A5A000F7E7404604B0BDE8F081D4E904300F89F4
:10A5B0000288498907FB02338A421BD2521C02805F
:10A5C0001A46616810E008886169072A088009D185
:10A5D000606801892069FDF737FF60682169C068FC
:10A5E00002F075FA2269616804B03046AC46BDE8F5
:10A5F000F04160470020D5E788DD070070B51C48B2
:10A6000001240168C90301D581130CE019480168D0
:10A610001522C9B2B2EBD10F07D10168C90704D026
:10A62000016801F0560101600024134D286A0128D9
:10A630001CD14FF4405011494068884208D123464C
:10A640004FF4805105F518706A6BFFF74BFE68B147
:10A6500000F09CFD014623460948AA69FFF742FE27
:10A6600020B101F0A7FB10F0B10000D0012070BDB7
:10A670000004004020050040D8750020DBE5B15102
:10A68000797800204169002901D0C06808477047E7
:10A690007047000010B50446801E062810D2DFE87F
:10A6A00000F00D03030F09090A494FF4702000F070
:10A6B000EDFA05E00120FFF76FFE01E000F0EAFF90
:10A6C00005484168002903D02046BDE810400847EE
:10A6D00010BD000089A907006859002010B5044684
:10A6E000062801D0072C02D1002001F06BF80448A5
:10A6F0000168002903D02046BDE81040084710BD7E
:10A70000A4590020BFF34F8F05480168054A01F4A2
:10A71000E06111430160BFF34F8F00BFFDE7000010
:10A720000CED00E00400FA052DE9FC4180461F46CF
:10A7300015460E4600240D4800F006FA38B11120E7
:10A74000BDE8FC8106EB043001F0E2FA641CAC4287
:10A75000F8D1064800F0F5F9CDE90057334600225C
:10A760000221404600F02AF80020E9E7F8590020CD
:10A770002DE9F843104D0F4680461E469146694626
:10A78000286800F0B2F9040014D01C21FDF75CFE2B
:10A7900001202071C4F81490380BC4F80080C4E97B
:10A7A00002606946286800F0C1F902F055FB0020FC
:10A7B000BDE8F8830420FBE7B4DB07002DE9F04394
:10A7C00087B00446DDE90E8980681D4616460F46AF
:10A7D00000280BD018216846FDF736FE02A88DF838
:10A7E000007080E86003A1686846884707B0BDE84C
:10A7F000F08330B50446006887B00D4680680028B5
:10A800001FD018216846FDF71FFE0195A06805902E
:10A81000207910B1012810D107E001208DF8000047
:10A8200020690290E068039005E002208DF80000A6
:10A83000E0680003029060690490206881686846BF
:10A84000884707B030BD0B2803D30B38C0B200F0E7
:10A8500009B870470249002208780A707047000062
:10A86000C0590020014908700B207047C0590020D2
:10A8700001490120087070476859002001490120F2
:10A8800008707047A05900200123723000F0FABF11
:10A890000EB59DF8080020F00F00401C20F0F000DD
:10A8A00010308DF8080068466DDF002819D19DF83A
:10A8B0000100401C8DF8010068466CDF002810D1B3
:10A8C0000848007A800703D50748011D806901E028
:10A8D00006A1072082B202A87CDF002801D105482A
:10A8E0007ADF0EBDA8590020605E002044667554D2
:10A8F0006172670046DA07002DE9F04781461D4680
:10A9000016468846494502D10020BDE8F087A8EBED
:10A910000900040B06F6FF704FF0000A070B00F069
:10A92000C3FAA5422AD22C4628E0A74202D8BA464A
:10A93000354601E0A246250300225146484600F074
:10A9400023FD0028E1D1681E00F003002A1A00232D
:10A9500041464846D21C00F02DFD0028D5D10948BB
:10A96000A7EB0A07761B016BA94429440163A8449D
:10A97000002000F013FF5FEA000AC6D1002ED4D1F8
:10A980005046C2E7D87500200120FFF705BD000042
:10A99000014941600020704788DB070010B50B4972
:10A9A00041600B4800F0D0F868B901F017FB084986
:10A9B0001C234FF4EE7208740448A1F5EE71001FD9
:10A9C000006800F07FF8002010BD0000B8DB070031
:10A9D000447F002002480068002800D00120704712
:10A9E000F85900200248007A002800D00120704762
:10A9F000447F002010B54FF44051144B4C6800F5D3
:10AA000000509C4204D042689A4201D1012200E0E9
:10AA100000229C4218D144689C4215D10A78142A1D
:10AA200001D9496900E00021094A0378B1FBF2F13C
:10AA3000142B01D9406900E00020B0FBF2F0814204
:10AA400001D0012200E00022104610BDDBE5B1512B
:10AA500040420F0070B5054608680C464A68866893
:10AA60002846314601F054FF6068286104F10C006B
:10AA70006861B0780221B1EB901F01D1241D2C61D7
:10AA800070BD000000F0E4F94FF48051002000F0A8
:10AA900011F940B90548C0F5FC2100F00BF910B9D7
:10AAA000034800F073F901F035FC00000080070056
:10AAB00091A6070010B5FDF7F8FB08B1002010BD06
:10AAC000112010BD10B531B1B2FBF3F403FB142417
:10AAD0001CB1092010BD0E2010BD01600021416095
:10AAE00081608281C381084610BD70B50C46054661
:10AAF000FDF790FB002802D021882868084470BD2B
:10AB000010B50A8849888A4203D1FDF7C5FB0120A8
:10AB100010BD002010BD70B50C460546FDF79FFB2B
:10AB2000002802D061882868084470BD10B50A88E2
:10AB300049888A4203D1FDF789FB012010BD00201E
:10AB400010BD002100F003B8012100F006B808B5DF
:10AB50006A46FDF7DCFB009808BD08B56A46FDF7BC
:10AB6000C9FB08BD38B5044600258DF8005068467D
:10AB7000FFF71EF921686268086890420ED9401EEE
:10AB800008600178238AE26801FB0325227A2168A4
:10AB9000101AC0B20A79824200D208719DF80000F2
:10ABA000FFF72AF9284638BD38B5054600208DF84C
:10ABB00000000C466846FFF7FBF8E868298A201A6F
:10ABC000B0FBF1F12A681068431C136001709DF816
:10ABD0000000FFF711F938BD10B530B1017A4268B5
:10ABE0000368891AC9B21A6006E00E2010BD036816
:10ABF0001A68541C1C601170491EC9B2F7D2006853
:10AC000000210171084610BD10B54FF0E0224FF051
:10AC1000FF314FF48054C2F88011C2F8801200F066
:10AC200005FC2046BDE81040AFF3008010B5044697
:10AC30001448C0F5FE2100F03DF808B1FFF730F8E8
:10AC400000F0A4FA014610488069421EC2F30B02CC
:10AC5000801A0144002001F6FF7100F02BF808B1C2
:10AC6000FFF71EF8D4E90001002282F3148882F372
:10AC7000108882F3118882F3138880F30888BDE876
:10AC80001040084700800700D875002070B5084DB7
:10AC900004460E46686802F0DFFC002C06D03246FF
:10ACA00021466868BDE8704002F0C8BC70BD000075
:10ACB00070590020F0B50A0502D1B0F5FE2F01D978
:10ACC0000720F0BD134D000B491E124F01222E1D0F
:10ACD000103700EB113407F1040C17E04309C3F1FE
:10ACE000000100EB411E02FA0EF106D0012B06D046
:10ACF000022B06D0032B08D105E0296005E0316066
:10AD000003E0396001E0CCF80010401CA042E5D916
:10AD10000020F0BD0006004070B5194D0024E86A1F
:10AD20002435012807D0A52808D0AA2809D0AC28A6
:10AD30000AD0002070BDFEF78DFF0BE002F00CF989
:10AD400007E0FFF773F805E002F006F908B9FFF72E
:10AD50006DF80124284600F03DFA0A4900200870E9
:10AD6000094800F01BFD08B1032070BD0120002C34
:10AD7000FBD00349096A0129F7D1022070BD000008
:10AD8000D8750020A05900207DA8070070B52A4D75
:10AD90006860002000F05CFC80BBFFF7BDFF20B1C5
:10ADA000012828D002283CD105E04FF47024FFF799
:10ADB00025FC10B932E04FF4A02400F075F81F4ACA
:10ADC00020211820FEF7DEFF08B1FEF769FF00F032
:10ADD000F1FF1621B1EBD00F09D100F0EBFFC00756
:10ADE00005D000F0E7FF164920F0B100086000F040
:10ADF00003FB18B903E00120FFF7CEFA11E0114977
:10AE00002046FFF743FF104800F0E0FA48B900BFC2
:10AE100000F036F8FEF796FF41DFF9E700F0C0FBDF
:10AE200008B1032070BD00202870084800F00AFC1B
:10AE3000FFF7EAFEF5E7000068590020205A0020DD
:10AE40001C05004089A9070095A6070071A8070006
:10AE500010B540F6F8700168491C02D1074900F0AE
:10AE60006FFF40F6FC700168491C05D1BDE8104039
:10AE70004FF4FC2100F064BF10BD0000008007000B
:10AE800010B501F04BF9002803D0BDE8104002F0E6
:10AE90004BBC10BD034A93680A46014698601846A9
:10AEA00002F0CCBB7059002070B50E4D28780028F8
:10AEB00017D101F033F9012690B10B480468A4F5CD
:10AEC0004864962C00DC962402F02EFC07492046AC
:10AED000FFF7E0FF4FF0E0214FF48030C1F80001B0
:10AEE0002E7070BDA15900200405014065D70700F0
:10AEF00040688068004710B542680830527900F019
:10AF0000F1F8002010BD2DE9F04399B01C469046A1
:10AF10000D460846DDF88090FFF7EAFF6E680746A9
:10AF20007079A04200D804462246414611A800F09C
:10AF300015F97279494601A800F0D4F801AB224610
:10AF400011A905F108000097FDF724FC18B10020B5
:10AF500019B0BDE8F08348F24250F9E770B51646E3
:10AF60000C46054600F0E2F800280ED1AA791946F1
:10AF7000304600F0E8F8002807D131462046FFF7B8
:10AF8000BAFF002801D10149216070BD7052464DC1
:10AF90002DE9F8430C46DDE90857814698461646E8
:10AFA0000D49204600F0B6F8002810D160683946F7
:10AFB00040794200284600F0C6F8002807D146B183
:10AFC00043463246214648460095FFF79CFFBDE8C0
:10AFD000F88348F21050FAE77052464D2DE9F041DF
:10AFE0001D46DDE906871646044600F02DF80028C8
:10AFF0000DD12A463146204600F03CF8002806D103
:10B000003A4641462046BDE8F04100F002B8BDE8AE
:10B01000F08170B515460E46044602F075FB002817
:10B0200007D13EB160682968C268914205D248F2F2
:10B03000145070BD48F2135070BD83682A463146E3
:10B040002046BDE87040184710B550B161B141606D
:10B05000096804468847002802D10548206000207E
:10B0600010BD48F2015010BD48F2105010BD000054
:10B070006E52464870B515460E46044602F044FB33
:10B0800000280BD146B155B160682A463146436865
:10B090002046BDE87040184748F2105070BD0020AF
:10B0A00070BD00002DE9F0410B480C4D0C4F401BCA
:10B0B000C60801203870002406E000BF55F83400AF
:10B0C0008047002805D1641CB442F7D302203870B1
:10B0D0000020BDE8F081000000000000000000003A
:10B0E000A259002070B514460D46064600F036F809
:10B0F000291930192246BDE8704000F02FB830B54C
:10B100000C46054600F035F828192146BDE83040C8
:10B1100000F02FB828B10068884205D048F24050AE
:10B12000704748F2105070470020704728B139B17D
:10B130000022C1E900201046704748F210507047C5
:10B1400048F21350704720B1914205D048F2115097
:10B15000704748F210507047002070470244521E5A
:10B1600004E000BF11F8013B02F801398242F9D234
:10B1700070470144491E05E002780B7800F8013B56
:10B1800001F801298142F7D2704700004FF4405086
:10B19000074A4168914207D18068411EC1F30B0103
:10B1A000401A00F6FF7070474FF48050704700005F
:10B1B000DBE5B15100B5FFF7E9FF054989690A18D8
:10B1C000401E0844C0F30B00101A00F6FF7000BDCB
:10B1D000D875002000210160416081600148016351
:10B1E00070470000D87500202DE9F0419846214FA6
:10B1F00016460C460546002301215BB1012B11D0F8
:10B20000022B1ED00020381AA0F50040A8421BD205
:10B2100001221AE0FFF7CEFF8EB11749096A012912
:10B22000F1D00CE0FFF7B2FFB8F1000F05D14FF4F9
:10B230004051124A4968914201D00121E3E70021BF
:10B24000E1E74FF48050DEE7002242EA0400884341
:10B2500005D0022B03D25B1CDBB2022BCCD912B17E
:10B260000420BDE8F0811BB103481830FFF7B2FF9E
:10B270000020F6E700800700D8750020DBE5B1511B
:10B2800070B504460078092811D2DFE800F01005F7
:10B2900010112510381013000D461D490320C968F0
:10B2A0008847606900F056FBFFF7CDFA687070BD03
:10B2B000084628E00D46A18A206900F027FBFFF729
:10B2C000C2FA68702846FFF787F8E1680029EED0D7
:10B2D0002069BDE8704008470C460D490831081F39
:10B2E00000F052FBFFF7AFFA60700128DFD10020B9
:10B2F00000F054FA0028DAD00A20607070BD0846C9
:10B300004FF40071C160BDE87040FFF765B8000000
:10B31000C459002070B51A4A05780124936C092D90
:10B320002CD2DFE805F02B052B0B0F2B252B08006B
:10B3300000F034FF22E000F0A7FF1FE08B60106DEB
:10B3400048601BE0D2E91454566C2C1BA64203D073
:10B3500008204870012411E00024556554642146FA
:10B36000D36400F055FF07490420C968884705E009
:10B370008B60106D48604FF48050C860204670BDEF
:10B38000D8750020C459002013460A4601460148DA
:10B3900000F0F0BB0C5A002008B1034900E003495B
:10B3A0000022034800F0FCBBC4DB070094DB07006D
:10B3B0000C5A002008B5009313460A46014602487D
:10B3C00000F086FC08BD00000C5A0020084910B5AA
:10B3D00008600020FFF782F9064800F00DFA002807
:10B3E00004D1BDE81040034800F026B810BD0000AD
:10B3F000A4590020DDA60700002070471FB589086A
:10B40000002201AB009283E80700684618DF04B011
:10B4100010BD00001FB5044B0FCB8DE80F00684630
:10B4200018DF04B010BD000048DB07004FF4805067
:10B43000410408600020704710B5040011D00120BD
:10B44000FFF7AAFF00280BD100F04EFA00F0DEFA59
:10B4500048B10949081F00F097FA012803D00320DA
:10B4600010BD072010BD04480838C4600020FFF755
:10B47000F9F9002010BD0000CC590020816819B1F5
:10B48000024A1821FEF70EBC0720704791B407004E
:10B49000AFF3008030B587B0044618221F496846D4
:10B4A000FCF7B9FF20788DF8000022781C4D0D2A9A
:10B4B00025D2DFE802F0240B270B0B240B240B24EE
:10B4C00024240700E968072088471BE020466946D6
:10B4D000062A01D0012A01D1027C2A702A78012A89
:10B4E00005D0022A06D000202870052008E0FFF7CA
:10B4F000C7FE07E0FFF70EFF20B907B030BD0220FE
:10B500008DF80100D4E90112684690479DF80100CA
:10B510000128F2D0E96805208847EEE770DB0700D4
:10B52000C459002038B10549016005494160012135
:10B530000172002070470E207047000045B50700DB
:10B540007DB5070010B50C0001464FF0110007D083
:10B550002278052A05D2DFE802F00F050D0F0F0053
:10B560000E2010BD084600F051F80028F9D1022144
:10B57000217010BD112010BD082010BD024608200A
:10B5800041B10B78022B04D1022A05D0032A00D145
:10B59000112070470E207047002003220A70704768
:10B5A00070B50B480024D0F82413491C03D1D0F8FF
:10B5B0006403401C09D04FF4FE25284600F0A8FB88
:10B5C000C9220349284600F0D3FB204670BD000085
:10B5D000D875002010B528B11C220349FCF71BFFC9
:10B5E000002010BD0E2010BD64F3070010B5064CFE
:10B5F00000221821201DFEF7F7FE2168814201D1AB
:10B60000012010BD002010BD64F3070070B50C4D83
:10B610000400D5F8640305F5597503D0401C03D028
:10B62000082070BD0E2070BD00221821201DFEF7DD
:10B63000DBFE206007222146284629DF70BD00007E
:10B6400000F00700014901F035BD000000F00700DF
:10B6500010B5FFF7A1FE30B900F01CF8002000F093
:10B660009DF8002800D0032010BD000010B5FF2277
:10B670004FF400710648FCF7E0FE0548202124380D
:10B68000FCF7E2FE024900205C39086310BD0000AF
:10B69000347600202DE9F0472E48FEF7C3FE2E4EEB
:10B6A000074634682046FEF7BDFE4FF0010A4FF012
:10B6B000000958B16068012806D02046FEF71AFE3E
:10B6C000D4F85C12884201D1012500E00025234C0A
:10B6D0004FF002084FF460719FB10A461D492046A1
:10B6E000FCF799FE9DB1366825465422311D281D70
:10B6F000FCF791FE4FF4327206F15C0105F15C003B
:10B7000003E015B30A4615483168FCF784FE60680B
:10B71000012818D11249402201F5E470FCF77BFEA4
:10B720000F491C22403101F5E470FCF774FE84F8E7
:10B73000609284F8A1A20B4884F8E292E169C0F813
:10B740002210C4F80480BDE8F0870448FCF77CFEB2
:10B75000F7E7000000F00700D4590020D87500205A
:10B76000347700205878002070B50546094801F06C
:10B77000ABFC084C20602046FEF7BCFDC4F85C0220
:10B78000A4F5E0632A462146BDE87040024801F076
:10B79000A0BC0000D875002000F0070070B5054679
:10B7A0000020FFF7E1FF040003D10349284601F020
:10B7B00081FC204670BD0000D87500204FF48050F9
:10B7C000704700002DE9F04107460948094D401B2C
:10B7D000C6080020044607E005EBC400416838466F
:10B7E0008847002802D1641CB442F5D3BDE8F0813B
:10B7F00084DE07007CDE07002DE9F041074609489A
:10B80000094D401BC6080020044606E055F83410D8
:10B8100038468847002802D1641CB442F6D3BDE8FC
:10B82000F081000084DE07007CDE0700012201F0C9
:10B83000CBB938B5144602780B467AB1012A04D048
:10B84000022A0DD0032A1BD112E0D0F801500022A9
:10B8500021461846FEF7C8FDA84211D1012038BD87
:10B8600001B02246BDE830400023401C00F00AB879
:10B87000411C40220020009400F0F2F80128EED094
:10B88000002038BD2DE9F041AAB0054620208846A9
:10B8900028901E4617460124782102A8FCF7D4FD03
:10B8A000FEF7D0FD2EB12022294620A8FFF756FC36
:10B8B00020AD28A90A48CDE900013B464246094986
:10B8C00002A8FFF78BFB28B9202229460448FCF781
:10B8D000C6FD00B100242AB02046BDE8F08100007A
:10B8E0002C7D002058D8070010B50648064C806B08
:10B8F00020B101F0D5FD08B1012000E0002020704A
:10B9000010BD0000D8750020D85900202DE9F04165
:10B910000F4C07460D46E06BA26B01264119914280
:10B9200001D9032610E00A492A465C310844394609
:10B93000FCF771FDE06B064A2844E063403229467B
:10B940003846FEF751FD20643046BDE8F081000026
:10B95000D875002070B504004FF0010504D0B4F58F
:10B96000007F03D9042508E0032506E004490020F0
:10B970000870FFF77BFE03488463284670BD000013
:10B98000D8590020D87500202DE9F04106461D4801
:10B990000F46C16B806B814201D008242FE01A4D05
:10B9A000287840B1FFF706FC30603946E86801F0BE
:10B9B0007FFE044623E001F073FDF8B100F02CF89F
:10B9C0000446002030603860012C0FD13946E86809
:10B9D00001F06EFE0446012808D1386801270021D5
:10B9E0003B460A46FFF700FC18B10424FFF73EFE71
:10B9F00005E0FFF7DFFB30602F7000E005242046F4
:10BA0000BDE8F081D8750020D859002001480078A1
:10BA100070470000D859002038B50F4C251D002074
:10BA200094F86C31014602463BB194F8D802B4F860
:10BA3000DA2204F5B87504F53771084B9C68009458
:10BA40005B6800F00DF8012804D1281DBDE83840DE
:10BA500000F050B838BD000058790020D8590020B7
:10BA60002DE9F041A2B0064620200D4620901F4649
:10BA70001446DDF8A080782102A8FCF7E5FC002040
:10BA80002190FEF7DFFC25B12EB1162022B0BDE8D3
:10BA9000F0811320FAE720A91448CDE900014346BC
:10BAA0003A46134902A8FFF799FA08B9402C01D089
:10BAB0000A20EBE70D48224629464038FCF7ABFC4C
:10BAC0000A4820214038FFF71AFB08484021403837
:10BAD000CDE90001A0F14801044A21A8209BFFF70D
:10BAE00057FA08B10520D1E70120CFE70C7D0020EF
:10BAF00058D8070070B5044690F85400012570B37B
:10BB000094F8550028B1012803D0022801D0032859
:10BB10002AD194F86E00032801D0142525E0207A5C
:10BB2000E8B1E068342801D011251EE0204601F07C
:10BB30005FFA68B1207898B194F855100C4849B173
:10BB4000012907D06168C06881420ED810250CE039
:10BB500012250AE061688068814206D2F6E703E0B8
:10BB600094F85500012800D00F25284670BD00002C
:10BB7000D87500202DE9F0410446406815461E4660
:10BB800002680F466A432046FEF708F820683346ED
:10BB90002A46D0F810C039462046BDE8F04160473B
:10BBA00001600B68114618472DE9F04128B1016882
:10BBB00019B1C969BDE8F04108470D4D0D48002491
:10BBC000461B14270DE000BF04EB840005EB80004A
:10BBD000016829B1C969884710B10120BDE8F08129
:10BBE000641CB6FBF7F0A042EED80020F6E7000098
:10BBF0000C5A0020205A0020044801214174007A88
:10BC000008B100207047012070470000447F0020E9
:10BC1000012801D0032808D10449002201284A74D0
:10BC200000D00020087401F0C9B87047447F00209C
:10BC300070B50146022801D0032943D1224C207A55
:10BC400000283FD0012831D002282FD11F480023DF
:10BC50000229006802D0032928D119E0E3600279A3
:10BC600012B1012A22D10BE0D0E90565721B142A1A
:10BC700000D314222A4482614569AA420ED015E0FD
:10BC80000169491C0161426991420FD1237213E09D
:10BC9000E268521CE260082A08D9E3602372022994
:10BCA0000AD00D21FEF7A5FD01F07EF8607C28B1D9
:10BCB000BDE8704000F098B90021F3E7BDE870409E
:10BCC00001F07CB870BD0000447F0020FC590020CA
:10BCD0002DE9F84304461D4616460F460846DDF892
:10BCE0002080FDF755FF3046FDF752FF2A463946C2
:10BCF0002046FDF753FFCDF8008020682B463246E2
:10BD0000D0F80CC039462046E047BDE8F883000073
:10BD1000094902220A60BFF36F8FBFF34F8F0A1DDC
:10BD2000106006480268002AFCD000200860BFF3BB
:10BD30006F8FBFF34F8F704704E5014000E401406F
:10BD4000094A01231360BFF36F8FBFF34F8F016068
:10BD5000064801680029FCD000201060BFF36F8FF7
:10BD6000BFF34F8F7047000004E5014000E401403D
:10BD700070B50E4C01232360BFF36F8FBFF34F8F5D
:10BD800000230B4D08E000BF51F8236040F823600A
:10BD90002E68002EFCD05B1C9342F5D3002020605F
:10BDA000BFF36F8FBFF34F8F70BD000004E50140FC
:10BDB00000E4014001480068C0B270471C05004023
:10BDC00008B5002242504058009008BD20B10349F8
:10BDD00009680160002070470E2070475CDD070095
:10BDE000FEB507460C460846FFF7F0FF002844D191
:10BDF000002500950195012606208DF80070ADF80C
:10BE0000040002958DF8026069462020226869DFEF
:10BE100000958DF801608DF80250019502958DF81E
:10BE2000035069464020226869DF00958DF8007054
:10BE3000F720ADF80200019502956946232022689B
:10BE400069DF0095019502958DF800606946012033
:10BE5000226869DF4FF4B060009001950295694651
:10BE6000A120226869DF0095019502958DF8006098
:10BE70006946A020226869DF0020FEBD60DF00283F
:10BE800002D1024A0121117070470000075A0020B8
:10BE900030B51548ADF5017D0078002821D04FF46C
:10BEA000FA7500BFADF8005280A9684661DF38B16D
:10BEB000052816D00DF5017DBDE83040FDF7F0BE38
:10BEC0006C460A497DA800F0BBF806E0D0E90021E5
:10BED000204690477DA800F0CAF87F980028E1D05E
:10BEE000F4E70DF5017D30BD075A002060DD070045
:10BEF000F8B5134C2078C0B10120A07001F0ACF867
:10BF0000112814D0022001F0BFF800258DF8005050
:10BF10006846FDF74DFF11DF064625709DF80000CD
:10BF2000FDF76AFF2EB13046F8BD0820F8BD0020AD
:10BF3000F8BDA57001F068FA032001F0A5F8F6E756
:10BF4000045A00207CB5194C207808B108207CBD2B
:10BF50000120A070002001F07FF8112819D00020E6
:10BF600001F092F812480026006801908DF80060F8
:10BF70006846FDF71DFF0F4901A810DF05000AD034
:10BF8000002020709DF80000FDF736FF2DB12846F7
:10BF90007CBD00207CBD0120F3E7A670667001F037
:10BFA00053FA012001F070F8F3E70000045A002072
:10BFB000F4DC07009D9C07000EB50749684600F0B9
:10BFC0003FF805E0D0E900108847684600F04FF8D8
:10BFD00002980028F6D10EBD10DD07000148007858
:10BFE00070470000045A00200548817819B1007894
:10BFF00018B1FFF77DBF08207047FFF7A3BF00000F
:10C00000045A00201FB568464BDF30B1052814D014
:10C0100004B0BDE81040FDF743BE084901A800F098
:10C020000FF806E0D0E900210098904701A800F041
:10C030001EF803980028E6D0F4E71FBD7CDD07005A
:10C04000016009684160AFF3008010B5D0E90021BC
:10C050005368994201D1002104E0D1E90034A342A0
:10C0600002D01946816010BD08314160F0E7816857
:10C0700000290BD0026892680A44826041684B68CC
:10C080009A4203D108314160FFF7DFBF70470000DB
:10C090002DE9F04104461348134BC01A0C21B0FBA4
:10C0A000F1F6A0694FF0FF3110F8022C02B92169B6
:10C0B000002011E000EB400503EB85052F68974257
:10C0C00009D14F1C02D06F688F4204D194E80F0051
:10C0D000AD68A84703E0401CB042EBD301202060CC
:10C0E000BDE8F081D4DE0700C8DE070010B51446B5
:10C0F00012680830202A02D248F2145010BD0022E3
:10C1000001F00FF80028F9D120202060002010BD98
:10C11000083001F08FB8083001F04CB902480068CF
:10C12000002800D0012070470004014030B587B0DE
:10C130000C460546182216496846FCF76CF9217B27
:10C1400014488DF800100195012906D0022915D058
:10C15000062917D1607B049014E08188C180607B40
:10C160000490617CD4F80E0061F31F600590049880
:10C17000012807D10848FFF725FB03E0B4F80D10AC
:10C180008180C1806846FFF779F907B030BD0000B3
:10C1900098DA0700A85900207CDE07002DE9F0415D
:10C1A0000C460546FFF732FC0826B8B16969032042
:10C1B00041B3154A154B0F0505D0576DD3F808C08C
:10C1C0000F4467451ED1B1F5805F01D9042019E005
:10C1D000506DD3F808C04718674502D96670BDE8AE
:10C1E000F0815164D16C10659164106369695A687B
:10C1F00001F6FF711044090B0022FFF7C5F8002873
:10C20000EDD005206070EAE7D8750020C459002001
:10C2100010B5044686B00020FFF7C6FC30B1154AC1
:10C2200018212046FDF73EFD06B010BD1822124928
:10C230006846FCF7F0F81148026D114881688A429F
:10C2400010D14068FFF7F2FA8DF80100FEF7FBFA13
:10C250008DF80100D4E90112684690470948FFF7BC
:10C260009DFAE1E701208DF80100D4E9011268464A
:10C270009047D9E711C2070058DB0700D8750020A6
:10C28000C459002009C307002DE9F0410E460446B9
:10C29000FFF7BCFB60B11A4DD5E91401401AA18A21
:10C2A0006A6C0844904205D903207070BDE8F081A3
:10C2B0000820FAE7134A286B52688718104A206949
:10C2C0004832FEF791F8D4E903318046A28A384615
:10C2D000FFF770F820B1D4E90310BDE8F04108473A
:10C2E000A18A286B08442863A18A286DC5F8488074
:10C2F00008442865C6F80880286D7060D6E70000FD
:10C30000D8750020C459002001490620C968084793
:10C31000C4590020BFF34F8F05480168054A01F456
:10C32000E06111430160BFF34F8F00BFFDE70000E4
:10C330000CED00E00400FA0501460148FEF734BCAC
:10C3400084DE070030B58A1D8B79083187B0022B57
:10C3500033D153888489A3422FD1127A012A2CD158
:10C36000184C0DF1040C3CCC8CE83C000A89ADF86B
:10C370000C204A890C3104911249ADF80E20803905
:10C38000114C096A0591CDF818D0018A05AA608878
:10C39000ADDF18B96846FDF7A1FF38B10020ADF850
:10C3A000080001A96088B0DF50B106E040F2FD103E
:10C3B000ADF8080001A96088B0DF002007B030BDEB
:10C3C0000120FBE7B0DA0700A8590020F8B50D46B8
:10C3D00014460646694600F057FA00280FD0009B25
:10C3E000B3F5803F0AD2981C834207D8A97802226D
:10C3F000B2EB911F02D02989814201D20020F8BD01
:10C400002380A11C3046009A00F074FBF8BD114651
:10C4100000F0D6B8114600F0E3B8F8B50C46154662
:10C420000646694600F030FA00280CD0009A501CED
:10C43000904207D3A1780223B3EB911F02D0218948
:10C44000814201D20020F8BD2946304600F052FB5F
:10C45000009A0021A954F8BD2DE9FF410C46CE6891
:10C4600017460546694600F017FB00280ED0E06825
:10C4700000280BD0A0783A46C0F3011002283146BC
:10C48000684606D000F0DAF80199696004B0BDE8AA
:10C49000F08100F086F8F7E77CB50D461446694652
:10C4A00000F08FF9002820D02889082806D0042819
:10C4B00009D002280AD001280CD015E0DDE90001DE
:10C4C000C4E900010AE00098206006E0009800B28C
:10C4D000208002E0009840B22070C117DDE90023FF
:10C4E00050405940084301D000207CBD01207CBD54
:10C4F0007CB50D461446694600F0A1F9002820D00D
:10C500002889082807D00021042809D002280AD049
:10C5100001280CD014E0DDE90001C4E9000109E0C4
:10C520000098206006E0009880B2208002E0009829
:10C53000C0B22070DDE9002350405940084301D0CB
:10C5400000207CBD01207CBD7CB50D4614466946AB
:10C5500000F075F9002821D02989082908D0009811
:10C56000C21704290BD002290DD001290ED014E0E6
:10C57000DDE90002C4E900020146134609E0C317E1
:10C580000146206005E001B2218001E041B2217046
:10C59000CB1741405340194301D000207CBD0120FE
:10C5A0007CBD70B50D46064614461146284600F07F
:10C5B0008EFA224629463046BDE8704000F03EB86B
:10C5C00038B50C460422694600F094FA002806D0DB
:10C5D0009DF80310009861F31F602060012038BDB2
:10C5E0001CB50C460822694600F084FA002824D0C5
:10C5F0009DF801109DF800209DF80230080E42EAD7
:10C60000012242EA034240EA13409DF803309DF8BC
:10C61000041040EA132008439DF8051042EA036223
:10C6200040EA01209DF8061040EA01409DF80710FD
:10C6300040EA0160C4E9002001201CBD2DE9F04F53
:10C6400004469DB000200090064601904FF0FF3A4E
:10C650000AA800F05DF94FF0010BE94682E012AB49
:10C6600005AA06A9204600F0C9F850B10AA8059904
:10C6700000F05FF960B10B98807810F0300F53D064
:10C6800060E09DF84800002870D11DB0BDE8F08F33
:10C690000598B04242D30B9D0AAE0B98807800F00B
:10C6A0000F00082812D0304600F05AF90B98A84223
:10C6B000F3D156460599B14230D3D4F80880099198
:10C6C0009DF8181008910E990D6820E00B980688C7
:10C6D000F0E729680F682FB1DDE9083229462046C6
:10C6E000B84711E011948968DDE908720988914220
:10C6F0000CD1294617A8FEF7ADF985F80CB017AA9A
:10C7000039461198FDF7FDFE0028BED0AD6815B181
:10C71000A1684145DDD0A168414523D19DF818109D
:10C72000204600F023FA1BE00C9840280AD200F0C3
:10C730001F010BFA01F00C994A0959F82230034302
:10C7400049F82230E5682DB10AAB9DF81820204643
:10C750000599A8470AAA9DF818102046FDF7D1FEB2
:10C76000002892D0A06800287FF479AFDDE90B049F
:10C7700085780AA800F0F4F80028F7D115F0300FFA
:10C7800003D10B98008800B1641CC4B10020494655
:10C7900005E000BF51F82020521C0ED1401CB0EB28
:10C7A000541FF7D3600959F8201004F01F00C0F19E
:10C7B00020022AFA02F0814201D0002065E7012020
:10C7C00063E71CB50C46694600F039F8002814D020
:10C7D000DDE90002C10709D051084FEA30006FEAD5
:10C7E00000026FEA0100C4E9002004E051084FEAAA
:10C7F0003000C4E900014FF001001CBDF8B5074648
:10C800000020187008700E4610601C4615466946D8
:10C81000384600F039F801004FF0010009D00099C6
:10C8200059B1C8082860009800F007003070012056
:10C83000F8BDB96809B10020F8BD2070FBE72DE90B
:10C84000F8430026884681463446354604E0402EAB
:10C8500002D30020BDE8F8836946484600F076F927
:10C860000028F7D09DF80070324607F07F00C10F16
:10C87000FBF7C2FD29430443F61D0D463806E6D4F6
:10C88000C8E900410120E5E7F8B50E4607466946CC
:10C8900000F05CF900280AD09DF80040200616D56B
:10C8A000072504F07F0403E0202D01D30020F8BD0C
:10C8B0006946384600F04AF90028F8D09DF8001083
:10C8C00001F07F00A8400443ED1D0806ECD40120D0
:10C8D0003460F8BD10B559680B4AC968914212D14D
:10C8E0000A4AD0E90110D2E90134234301D00020E3
:10C8F00008E011F8013BA0F101001B06F9D4C2E9E0
:10C9000001100120907010BDE0D80700D859002018
:10C91000C26000230160C0E901138B881A440261E0
:10C92000B1F906301A4442610888002800D001207D
:10C93000704770B545680E46044660680188B1428C
:10C9400006D1807800F00F00082801D0012070BDCA
:10C95000204600F005F86068A842EED1002070BDC6
:10C9600030B541680A885AB101F1100343600A8A60
:10C9700042B18C780A89C4F30115032D07D00BE06E
:10C98000002030BDC2680168FFF7C2FFF8E79D785C
:10C99000C5F30115032D06D00225B5EB141F08D1F0
:10C9A0004C89624309E08D8804690022641B04619C
:10C9B00003E0B5EB941F00D10422897811F0300F09
:10C9C00002D18168491C81609C880169214411441D
:10C9D0000161B3F9062011444161012030BD30B539
:10C9E0004168002487B0897801F00F02082A11D02D
:10C9F0008A091ED00222B2EB911F09D10269C1F34C
:10CA000001110229146001D0032901D14069048079
:10CA100007B030BD0069056808E02C7329466846F8
:10CA2000FEF718F86846FFF7DAFFAD68002DF4D17D
:10CA3000EEE7C1F30111012912D00229E6D0032942
:10CA4000E4D04268917801F00F0107290BD0D1683A
:10CA500081B11289006907B0BDE83040FBF7DBBC4B
:10CA600041690C70EDE70169D06807B0BDE830405E
:10CA700000F02DB81189006907B0BDE83040FBF720
:10CA8000E3BC000010B5034B002408C080E816008A
:10CA900010BD0000BDA3070038B50D460446694629
:10CAA000FFF7F2FE00280BD0D4E90002D4E902130C
:10CAB000C5E90002C5E902130098814201D20020B5
:10CAC00038BDA860A168081AA060012038BD00B573
:10CAD0000A4687B001466846FFF71AFF002807D0CC
:10CAE0006846FFF77CFF6846FFF73AFF0028F7D15A
:10CAF00007B000BD7FB514460546A9B9124A28689B
:10CB0000904208D110E0102269462846FFF7F2FF54
:10CB1000002807D0103C102CF5D82246694628463C
:10CB2000FFF7E8FF04B070BDA868A04201D2002062
:10CB3000F8E72B682246284698470028F2D0A868D4
:10CB4000001BA8600120EDE7BDA3070010B5044657
:10CB50008068002809D023680122204698470028D1
:10CB600003D0A068401EA060012010BD38B500248D
:10CB700039B1012912D0022912D005291DD0002077
:10CB800038BD0546012269462846FFF7B3FF90B13C
:10CB90009DF800000006F5D4012038BD08220DE004
:10CBA00005466946FFF770FE28B100212846009A25
:10CBB000FFF7A0FF38BD204638BD0422BDE838404D
:10CBC0000021FFF797BF00002DE9F04F81462C4868
:10CBD00017460E46C5680A4693B0012449462846C2
:10CBE000FDF752FEDFF89C80A24670B195F8550023
:10CBF00068B100F00101C0F340024B462846CDE980
:10CC0000006700F043F8D8B11BE0172419E0CDE924
:10CC1000006A4B460022294602A8FDF771FB4FF03F
:10CC2000000B68B10FB3412202A91748FBF7F3FBD1
:10CC3000C8F820B0C8F82CA06968C8F8081017E038
:10CC400005246FB1012C13D00E482430FEF7C2FA30
:10CC5000FEF70CFDC8F8489013B02046BDE8F08FF1
:10CC6000012C02D0FEF702FDF6E7C8F814A0F3E7A6
:10CC7000002231464846FDF7B7FBC8E90960E7E7FF
:10CC8000D8590020D8750020797800202DE9F04788
:10CC9000A4B08946DDE92C5A04469846164644213C
:10CCA00002A8FBF7D1FB442113A8FBF7CDFB4746B5
:10CCB000B9F1000F38D008F50050384A4368A16D2B
:10CCC000934255D14B1EC3F30B03C91A41F6FF73B0
:10CCD000D0F808C019448C454AD34FF440514B68F2
:10CCE00093420DD10A78102A01D9096900E0002188
:10CCF0000278102A01D9006900E00020814237D172
:10CD00004046FDF777FE00B18EB30121A06DCDE95D
:10CD1000000143460022214602A8FDF7F1FA00284F
:10CD200027D0A06D07442D1A56B10020CDE9005040
:10CD30003B464A46214613A8FDF7E2FA002818D0E0
:10CD4000BAF1000F28D0164DB9F1000F19D04046A6
:10CD5000FDF750FE18B105F11800FEF73BFA41222D
:10CD600002A91048FBF757FB36B1AC2005E0FFE7FE
:10CD7000002024B0BDE8F087A520E862A06D6863BC
:10CD800001E0AA20E8623EB10648412213A98230A0
:10CD9000FBF741FB6068E8600120EAE7DBE5B151A1
:10CDA000D875002038780020034802490068FDF754
:10CDB000A7BE0000005A0020B4DB07002DE9F041B7
:10CDC000224C0025224E207A012730B92148311DFE
:10CDD0000068FDF7A0FE306038B102202072316893
:10CDE000087928B101281BD113E06560BDE8F08106
:10CDF000D1E90503C01A142800D31420820806D0F4
:10CE000082080869C9681844194429DF05E001222D
:10CE1000F7E7D1E90301084428DF58B1112812D0FF
:10CE200003213068FDF7E5FC25726560BDE8F0413F
:10CE3000FFF7BABF207C0028D8D1BDE8F04100211F
:10CE40000220FEF7F5BE2772D0E70000447F0020E5
:10CE5000FC590020B4DB070010B5074C201DFDF77E
:10CE600073FE002806D1607C002803D1BDE8104085
:10CE7000FFF7A4BF10BD0000447F002010B510468E
:10CE80001A46FBF7C8FA002010BD10B510461A4626
:10CE9000FBF7C1FA002010BD2DE9F0411E681C46C9
:10CEA0001546074621B1012918D0052923D119E0DB
:10CEB00000202060401C2060B0421CD8012229467E
:10CEC0003846FFF717FE002806D015F8010B0006BC
:10CED00001D52068EEE70120BDE8F0810820024678
:10CEE000186002E004200246186029463846BDE872
:10CEF000F041FFF7FFBD0020EEE770B516460A4689
:10CF00000446C11C104600F0B1FB054661193046CD
:10CF1000C91C00F0ABFB284470BD000003B5094AF2
:10CF200085B0D2E91612CDE9001207498989ADF81A
:10CF3000001006A9CDE90210044869464088AEDF1A
:10CF400007B000BD30DA07007C5E0020A859002041
:10CF5000084670470846704770B5FEF72FFC114A27
:10CF6000114E136B546B916CE21A551EC5F30B05F1
:10CF7000521B42F2040518446D5802F6FF72B54286
:10CF800001D0032070BD1944A34201D1002070BD1F
:10CF90000823FDF7B1FC0028F9D1BDE87040FEF789
:10CFA000FDBB0000D8750020DBE5B151F0B50546AA
:10CFB000002003464FF440540C4E4FF6FE7712E02B
:10CFC000D4F804C0B44505D155F823C0B4F80CE03A
:10CFD000F44504D02AB155F823C0BC4501D1012045
:10CFE000F0BD5B1CDBB28B42EAD3F0BDDBE5B15197
:10CFF00010B54FF44051174B4A68018A9A4221D12B
:10D0000071B100F11403426990F8550062B104282F
:10D0100008D00022BDE81040C9B21846FFF7C6BFCD
:10D02000002010BD0122F5E710B1012808D1F7E773
:10D03000012905D9C9B200221846FFF7B7FFEFE76B
:10D04000012010BD11B141690029E9D10078002803
:10D05000F6D110BDDBE5B1513EB50446094968463D
:10D06000FEF7EEFF08E000BFD0E900212046904720
:10D0700030B16846FEF7FBFF02980028F4D13EBDB0
:10D0800011203EBDF8DC07003EB50446084968465D
:10D09000FEF7D6FF07E000BFD0E900212046904709
:10D0A0006846FEF7E4FF02980028F5D13EBD000077
:10D0B00004DD070002460348014B006800F009B890
:10D0C00058720020D459002000225821001DFDF77D
:10D0D0008BB92DE9F04114464FF460751E460F469A
:10D0E00080462A46FBF7BBF930B1002201214046B9
:10D0F000FEF74AF998B905E00CB10020A0470020DE
:10D10000BDE8F0812A4639463046FBF784F92346CC
:10D110002A4631464046FEF74DF90028F0D003205C
:10D12000EEE770B516460D46040007D035B1206C09
:10D13000802200213828225403D307E00E2070BD3E
:10D140002154401C3828FBD30BE02154401C4028BC
:10D15000FBD32146084600F097F838212046FBF71C
:10D1600073F9216CD4E912304A0FC90038345918C8
:10D170005041C4E90410227CE2710A0A42EA0062CA
:10D18000A2710A0C42EA00426271020242EA116094
:10D1900020716069E070010AA170010C6170000EDD
:10D1A00004F838092146084600F06EF84FF00002F6
:10D1B000EEB1E06ED100C840A854A36ECB40A818D1
:10D1C0000371636ECB400372236ECB400373E36D38
:10D1D000CB400374A36DCB400375636DCB400376E6
:10D1E000236DCB40521C0377042AE2D31FE018239F
:10D1F0005042216D03EBC000C140A954666DC6408A
:10D20000A9180E71A66DC6400E72E66DC6400E736B
:10D21000266EC6400E74666EC6400E75A66EC6407B
:10D220000E76E66EC640521C0E77042AE0D300202C
:10D2300070BD0000A8B100210164C0E912110A49C3
:10D2400001650A4941650A4981650A49C1650A497A
:10D2500001660A4941660A4981660A49C166002099
:10D2600070470E207047000067E6096A85AE67BB0D
:10D2700072F36E3C3AF54FA57F520E518C68059BB8
:10D28000ABD9831F19CDE05B2DE9F04FC8B0002268
:10D2900013466F46CC181B1D2568E4782DBA25F07F
:10D2A000FF05254347F82250521C102AF2D31BE0F9
:10D2B00007EB820151F8083C4FEA734484EAF344D7
:10D2C00084EA932451F83C3C4FEAF31585EAB345D0
:10D2D00085EAD303234451F81C4C51F8401C2144E7
:10D2E000194447F82210521C402AE1D3036D47939A
:10D2F000416D4691846D4594C26D44929246026E92
:10D300004392456E4295A946856E4195C66E4096FC
:10D31000B34600264FEAB21787EAF22787EA726C13
:10D3200002EA090725EA020887EA0807BC44204FF9
:10D3300057F8268008EB0B07BC445DF82670AB4617
:10D340000CEB070E4FEAB30787EA733787EAB35C43
:10D3500081EA04074D4601EA040891461F400AEBA2
:10D360000E02A24687EA08070C46BC441946761C02
:10D370000EEB0C03402ECDD3479E33440365469BF2
:10D380001944416545992144816544995144C165D9
:10D39000439911440166429949444166419929449F
:10D3A000816640995944C16648B0BDE8F08F0000DD
:10D3B000E4DB07002DE9F04116460F46040004D0D7
:10D3C00006B317B10025A8461AE00E20BDE8F0818B
:10D3D000216C785D6054206C401C206440280ED184
:10D3E00021460846FFF750FFD4E912014FF40072BE
:10D3F000801841F10001C4F84080C4E912016D1C9D
:10D40000B542E5D30020E1E710B51620FCF7AEFBEE
:10D4100048B10C4882684FF4800152B1016821F490
:10D420008001016010BDBDE8104042F20100FCF730
:10D4300037BC4FF0E020C0F88011BFF34F8FBFF32F
:10D440006F8F10BD4C7D002010B51620FCF78EFBB1
:10D45000A0B1114890F800044009082811D2012118
:10D46000814011F0EC0F0CD00C4882684FF4800121
:10D470006AB1016841F48001016010BD42F201000F
:10D4800001E042F20200BDE81040FCF709BC4FF099
:10D49000E020C0F8001110BD16E000E04C7D002037
:10D4A0007FB52A4800F15C01826B6846FFF7EAFA13
:10D4B000274E9DE8070006F11C03274C83E8070070
:10D4C00019462448C8600020A0706060A0604FF436
:10D4D0004771A6F54070FAF7B7FFA6F540721F49ED
:10D4E00002F54770FFF75DF800282BD0A07858B3FD
:10D4F000A6F5407090F86C11002901781CD019BB7A
:10D5000090F8720100B3D4E90112A6F5C675684619
:10D51000FFF7B8FA9DE80F001C3686E80F004FF4BD
:10D52000B2712846FAF790FF2A460D493046FFF7B8
:10D5300038F8002806D003E031B1807920B1094DD8
:10D540000120E56004B070BD0020FBE7D875002025
:10D55000587C0020D5C80700D859002000DA070001
:10D56000E0D807006079002070B503466FF07F4077
:10D57000814200D20846124DD5F804250244081A0B
:10D58000411E22F07F425860952902D29630963A89
:10D5900058601C7B05EB8400C0F8402509494FF416
:10D5A000F86088474FF4A07000EB84012846FEF72E
:10D5B00007FC4FF48030A040C5F8040370BD0000A4
:10D5C0000040024051D8070070B5174E307800284F
:10D5D00029D1164800680125C0F3004008B9144855
:10D5E0000560144C4FF480712046FEF7E9FB4FF4C0
:10D5F000A0712046FEF7E4FB4FF4A2712046FEF72F
:10D60000DFFB0D49A02081F800040B4910202039D0
:10D61000C1F800010020C4F80805A56025600220BB
:10D62000C4F80403357070BD705900201804004020
:10D63000080000400040024024E000E070B51546BC
:10D640000E460446FFF7C0FF314620462560BDE880
:10D650007040FFF789BF0000017B4FF480308840A5
:10D660000149C1F808037047004002400870020AEF
:10D670004A70020C8A70000EC870042070470000C7
:10D6800010B50248FDF75DFA002010BDF8590020E2
:10D6900010B514210448FAF7D7FE04480068FDF7D6
:10D6A00009FA002010BD0000447F0020B4DB070011
:10D6B00030B50F2490F8553000220BB1042B03D164
:10D6C00090F86450012D06D0DD0707D090F8565031
:10D6D000012D02D002E0826E0DE0826D9B070AD51B
:10D6E00090F85C30012B06D1064B006EC3F5FC238D
:10D6F000984205D802440AB101240A60204630BD90
:10D700000424FBE70080070030B100680549884227
:10D7100005D048F20250704748F20150704700208F
:10D72000704700006E52464870B5FEF7F7FC0028BF
:10D7300011D00020084A094B094C0121166801FA52
:10D7400000F52E4203D004EB8005C5F80036401CDE
:10D75000C0B20728F2D370BD080501403546526EAD
:10D7600000000140FFF7E0BF002070470020704735
:10D770002DE9FC4180461C4617460E460C48089D84
:10D78000FDF7E2F910B11120BDE8FC81A20839468D
:10D790003046FEF7EDFA0648FDF7D3F933463A4630
:10D7A00001214046CDE90045FDF708F80020EBE7F0
:10D7B000F85900202DE9F84F114D884681461E4644
:10D7C00017466946DDF828A02868FDF78EF90400A1
:10D7D00013D01C21FAF738FE00202071C4F8009005
:10D7E000C4E90486C4E902A769462868FDF79EF9E2
:10D7F000FFF732FB0020BDE8F88F0420FBE70000B4
:10D80000B4DB07007EF8C9F6120F4CD79208C1713D
:10D8100083F5768FE216ECBA29939A7403F32B06FC
:10D820009BFC932EF7111725792DB9D6BE74B76CD2
:10D830006731C8341D64FD04B795B1DC017F21F167
:10D84000461AF08B000000000000000000000000FD
:10D850000338FDD87047000011C1070017C1070049
:10D86000EDC007002000000078000000000000006C
:10D8700048002800002040008D87070000000000BD
:10D880000100010000000000010000000000000095
:10D89000020005000100000022000000000000005E
:10D8A0000000000000000000000000000000000078
:10D8B0000100010000000000010000000000000065
:10D8C000020005000100000042000000000000000E
:10D8D0000000000000000000000000000000000048
:10D8E000010011000400FCFF040000000000000023
:10D8F000020011000400FCFF040000000000000012
:10D90000030021000400FCFF0400100000000000E0
:10D91000040011000100FFFF0100000000000000F2
:10D92000050011000200FEFF0400000000000000DE
:10D93000060011000400FCFF0400000000000000CD
:10D94000070011000400FCFF0400000000000000BC
:10D95000080017000200FEFF2400000080D8070026
:10D96000090010000100FFFF010000007CD8070043
:10D970000A0027000200FEFF44000300B0D80700A1
:10D980000000000000000000000000000000000097
:10D99000010011000100FFFF010000000000000075
:10D9A000020017000200FEFF64010000E0D807003B
:10D9B0000000000000000000000000000000000067
:10D9C00001000700000000006801000090D9070076
:10D9D0000200010000000000010000000000000043
:10D9E00003000500010000004200000000000000EC
:10D9F0000000000000000000000000000000000027
:10DA0000010017000400FCFF6801000090D9070026
:10DA1000020017000400FCFFAC010000C0D90700A1
:10DA200000000000000000000000000000000000F6
:10DA300000110300001113000200000001000000AB
:10DA40000338FDD870470C000C000000580200009D
:10DA500002000000000000000200000000000000C2
:10DA6000405E0020090000000000000000000000EF
:10DA7000010000000000000028000000000000007D
:10DA80000000000000010000000001000000000094
:10DA90000000000000000000000000000000000086
:10DAA000559F07000000000000000000000000007B
:10DAB0000200000000000100000000000000000063
:10DAC0000800000000000000559F070039C3070050
:10DAD0000000000000000000040000000000000042
:10DAE0000000000000000000000000000000000036
:10DAF0000000000000000000000000000000000026
:10DB0000F400000000000000180000000000000009
:10DB10000000000000000000000000000000000005
:10DB200000000000000000000000000000000000F5
:10DB3000170000000000000050EADA308883B89F28
:10DB4000604F15F30000C98E0200000000000000C5
:10DB500000000000000000000400000000000000C1
:10DB600000000000000000000000000000000000B5
:10DB700000010000000000000000000000000000A4
:10DB80000000000000000000001000000400000081
:10DB90000100000091A9070081D607007DCE070093
:10DBA00071D7070029A7070051CF070069D70700E1
:10DBB000D5A90700587D00200010000004000000D7
:10DBC000010000009DA9070091D607008BCE070039
:10DBD000B5D7070071A7070055CF07006DD707001D
:10DBE000E5A90700982F8A4291443771CFFBC0B551
:10DBF000A5DBB5E95BC25639F111F159A4823F9218
:10DC0000D55E1CAB98AA07D8015B8312BE85312470
:10DC1000C37D0C55745DBE72FEB1DE80A706DC9B31
:10DC200074F19BC1C1699BE48647BEEFC69DC10FDD
:10DC3000CCA10C246F2CE92DAA84744ADCA9B05C19
:10DC4000DA88F97652513E986DC631A8C82703B0DC
:10DC5000C77F59BFF30BE0C64791A7D55163CA06EA
:10DC600067292914850AB72738211B2EFC6D2C4DF6
:10DC7000130D385354730A65BB0A6A762EC9C281E4
:10DC8000852C7292A1E8BFA24B661AA8708B4BC27A
:10DC9000A3516CC719E892D1240699D685350EF4A4
:10DCA00070A06A1016C1A419086C371E4C7748275B
:10DCB000B5BCB034B30C1C394AAAD84E4FCA9C5BD1
:10DCC000F36F2E68EE828F746F63A5781478C88422
:10DCD0000802C78CFAFFBE90EB6C50A4F7A3F9BE04
:10DCE000F27871C6A0DE0700A8DE07000000000081
:10DCF0000000000000100201E4DC0700F4DC070073
:10DD0000080000001CDD07002CDD070008000000F3
:10DD10002CDD07003CDD070008000000C0DE070026
:10DD2000C8DE07000000000000000000B0DE0700B1
:10DD3000C0DE07000000000000000000000000003E
:10DD400000000000000000000000000098DE070056
:10DD5000A0DE07000000000000000000685900205D
:10DD60003CDD07005CDD070008000000A8DE0700BE
:10DD7000B0DE070000000000000000006CDD0700BE
:10DD80007CDD07000800000049C50700F1C407005A
:10DD900099C407000FC4070015C40700CDC30700CE
:10DDA0001BC4070059C40700000000000820000140
:10DDB000FFFFFFFFFFFFFFFFFFFFFFFF000000006F
:10DDC000000000000000000001000000FFFFFFFF56
:10DDD000512563FCC2CAB9F3849E17A7ADFAE6BC0D
:10DDE000FFFFFFFFFFFFFFFF00000000FFFFFFFF3F
:10DDF00096C298D84539A1F4A033EB2D817D0377E5
:10DE0000F240A463E5E6BCF847422CE1F2D1176B7F
:10DE1000F551BF376840B6CBCE5E316B5733CE2B52
:10DE2000169E0F7C4AEBE78E9B7F1AFEE242E34F81
:10DE30004B60D2273E3CCE3BF6B053CCB0061D65BE
:10DE4000BC86987655BDEBB3E7933AAAD835C65A47
:10DE500039860700CF960700E5940700D4DE070057
:10DE600068590020B80000004C9B07008CDF0700B9
:10DE7000205A0020383500005C9B07006DA0070089
:10DE80000DA00700B8590020905E0020A15E002080
:10DE9000A45E0020F400000005A1070000000000BF
:10DEA000F9BB07000000000031BC070000000000C3
:10DEB00091BE07000000000005C007000000000040
:10DEC00011BC07000000000000000000030000007B
:10DED00025B5070000000000000000000000000061
:10DEE0008059002090590020000000000000000030
:10DEF0000000000000000000000000000000000022
:10DF00000000000000000000010000000000000010
:10DF100000000000FF00FFFF000000000000000004
:10DF200000000000000000000000000000000000F1
:10DF300001000000000000000000000000000000E0
:10DF400000E00700000000000000000000000000EA
:10DF500000000000000000000000000000000000C1
:10DF600000000000000000000000000000000000B1
:10DF7000000000000090D00300000000000000003E
:0CDF800085A6070000100000000008004B
:020000041000EA
:041014000080070051
:020000041000EA
:0410180000E00700ED
:04000005000782016D
:00000001FF
